:020000020000FC
:10000000B8CDA5C10000000020C0000089C00000DC
:10001000000093C00000000000000000020304067E
:10002000080C10182030406080000406080C1018DE
:100030002030406080A0C0000003070F1F000D0D9E
:1000400004050D050205030302004FB662FD0CC056
:10005000552041F00994C52DC095089483FDC7959E
:10006000C4BD64604FBE1895C0916400089483FDC0
:10007000C795C4BD6B7FC0916400CF3F09F419C020
:100080004FBE9098919893981895909891989398BE
:1000900076FD0DC064FD0BC0C9E0CA95F1F7C091B3
:1000A000B100C0FD959AC1FD979AC2FD949A4FBECA
:1000B000189524BCCC27C064C8BF6460F8CFCBCFF0
:1000C00070FFC9CF64FDC7CF909AC5CF70FFC3CF73
:1000D00064FDC1CF919ABFCF70FFBDCF64FDBBCF90
:1000E000939AB9CF959870FFB6CF64FDB4CFCEE1A7
:1000F000CA95F1F7909AAFCF979870FFACCF64FD97
:10010000AACFCEE1CA95F1F7919AA5CF949870FF46
:10011000A2CF64FDA0CFCEE1CA95F1F7939A9BCF11
:100120004FB6C9B7CF7EC9BF6E7FCCB5CE0DDDB59A
:10013000DF1DDBBDCABD4FBE18953FB68F7EABB786
:10014000A074A2118061A0E0ABBFA9B7AE7FA9BF28
:100150007894A0916800AA2341F085FD2EC0A0915B
:100160006800AA95A093680028C040E050E085FD93
:1001700014C0A0B396FDA095A2FD4FEFA3E096FD9D
:10018000A2E0A5BFAA27A064AABF8D7FA0B396FD59
:10019000A095A2FD5FEF451741F7A8E161FDA0938F
:1001A000680085FD03C0A8E1A09368004093960015
:1001B0008160442311F02092990085FD0EC0A0912A
:1001C0006900AA2331F0A0916900AA95A093690063
:1001D00004C08061AA27A064AABF80FF3CC0A09190
:1001E00096004A2F61FF8E7F85FD1CC0A091B40050
:1001F000A430C1F4403F08F040EFA42FA295AF70A7
:100200004A0F5091B600533069F0A695A69550FD5F
:1002100001C0A69552FD03C0A41B4A2F03C04A0F7C
:1002200008F44FEF40936100A72FA670A1F073FD73
:1002300012C0A0917000AA0FAA0F50919E0056956F
:100240005695541708F0452F4A0F4093610018F453
:10025000AFEFA09361004091B400443009F03AC080
:10026000A0916100A093630040916300A0919B0066
:100270004A1708F04A2FA0919D004A1708F04A2F0C
:10028000542EA091A000AA2309F422C0542F5A1B77
:1002900010F4A42F50E0BA2E8894AA1FAA2EA09181
:1002A000A200A095AA22A50E58F0A091A100A21527
:1002B00009F0AA95AA0EA093A10048F04A2D08C003
:1002C000A091A100BA1608F0A395A093A1004FEF4A
:1002D00040936400A0916000A395A093600051F04A
:1002E000F894A9B7A160A9BF84FF02C0A0E4ABBF86
:1002F0003FBE1895A0917400A395A093740041E0AF
:1003000050916800552329F085FF03C05A955093FA
:100310006800A0919600A13018F0209299000DC0BD
:1003200020929A002092A300A0919900AF5FA09321
:10033000990018F0AFEFA0939900F894A9B7A160C5
:10034000A9BF84FF02C0A0E4ABBF3FBE18953FB673
:100350004CB55DB58F7EABB7A074A2118061A0E0F3
:10036000ABBFA9B7AE7FA9BF789481FD23C0A2E03F
:1003700096FDA3E0A5BF8260A0B396FDA095A2FF65
:1003800005C040936500509366003EC1A3E096FD12
:10039000A2E0A5BFAA27A064AABF8D7F85FF01C0E8
:1003A00026C140E0A0B396FDA095A2FD20C14093D8
:1003B00096000FC1A3E096FDA2E0A5BF8D7F61FF6F
:1003C00071C0A2E096FDA3E0A5BFAA27A064AABFC2
:1003D00082604093910050939200A0908F004A1940
:1003E000B09090005B09BB24A22C4C38520518F445
:1003F0002092950049C0A091D400AA2359F1483C0D
:10040000520528F4A0E1BA2EAAE0AA2E23C048364D
:10041000A1E05A0728F4A8E0BA2EAFE0AA2E1AC02D
:10042000403DA2E05A0728F4A4E0BA2EAEE1AA2E7D
:1004300011C0403AA5E05A0728F4A2E0BA2EACE376
:10044000AA2E08C04839A8E05A0720F4A1E0BA2E25
:10045000A8E7AA2EC42EA0919300CA1AD52EA09167
:100460009400DA0ADD202AF4AFEFC094D094CA1ABF
:10047000DA0A20929500A8E0A210A0E0CA14DA06D9
:1004800018F4A1E0A093950040939300509394003A
:10049000409191005091920040938F0050939000B2
:1004A00042E097C0A09165004A1BA09166005A0BDC
:1004B00094FD82C093FD80C092FD7CC086FF03C086
:1004C000D52EC42E0CC05695479591FD73C05695F8
:1004D000479590FD6FC0D52EC42ED694C79461FD6C
:1004E00019C0AC2DAC51AD2DA24008F005C0DD20E7
:1004F00089F4AC2DA85C70F4A0916700A395AA23A1
:1005000011F0A0936700AA3008F471C02092960001
:1005100081606DC0A0916700AA2319F0AA95A093ED
:100520006700A22C5091BA0097FD06C0A090C800A9
:10053000533011F4A090D000AAEFAA0EA22DA21D54
:10054000CA18DA0A4FB74170533049F4442321F0F6
:1005500087FD05C0806803C087FF01C08F774423F3
:1005600059F0533031F4AFEFC094D094CA1ADA0A7C
:1005700003C040E050E020C0533049F4CC0CDD1CF7
:10058000AAE0CA1AD20818F4A0E0CA2ED22CAFEF03
:10059000CA16D20418F04FEF50E00EC0A091AC0084
:1005A000CA9E412D000C441F50E008F012C04FEFCE
:1005B00050E00FC05695479594FF07C0552309F0AA
:1005C0004FEFA42FA6954A0F521D4F3F520508F03A
:1005D0004FEF40939600816061FF09C0AFE1A095A5
:1005E000A923AB299A2F8F7DBB2009F48062A8E153
:1005F000A093680085FF03C0AAE0A093680061FD96
:1006000003C085FD01C08F7E85FD03C0A6E0A093D9
:100610006900F894A9B7A160A9BF84FF02C0A0E453
:10062000ABBF3FBE189511E00AC013E008C01AE046
:1006300006C01EE104C014E602C018EC00C005E1CB
:10064000BB27BA95F1F70A95D9F71A95C1F708951E
:100650002AE338E709C020E33CE806C02AE234EB8D
:1006600003C025E238EC00C0B091AD00BA9509F4A2
:10067000089512E0BB279798BA95F1F7919ABA9529
:10068000F1F79198BA95F1F7979ABA95F1F7123078
:1006900009F0909A123009F4939AB091AD00BA958E
:1006A000F1F7123009F09098123009F49398B7E8F6
:1006B000BA95F1F71A95F1F6022FB22FBA95F1F724
:1006C0000A95D9F73A9581F697980895221B39E053
:1006D000001F3A9509F40895221F211B18F4210FD9
:1006E0008894F6CF0894F4CF622C722CB0E08894F2
:1006F000B395221F331FE0F7379527958894912EE5
:10070000802E020B130B10F4192D082D10F4889471
:1007100001C00894661C771CBA9571F7172D062D39
:100720000895322D11232AF43A9500951095031B54
:10073000130BF894029F712C002D129F912C802C8A
:100740007894780C172D921C292DB4E06B2E2695E9
:10075000179507956A94D9F7332321F000951095E2
:10076000031B130B08950091B4000430A1F1B09164
:100770009600B15008F010C0B0916100B0936300D2
:1007800020927E0020927F002092800020928100A3
:10079000209282006F7D1FC06090B4006062B091B3
:1007A0006100B093620008E317EC20917A00309169
:1007B0007B0036952795B62DBA9541F0369527954D
:1007C000B62DBA95BA9511F0369527958DDF009321
:1007D0007E0010937F00089500917E00B09162002A
:1007E0000B1B10917F00120928F40038BFEF1B0784
:1007F00040F009C00F37120508F405C00FE710E0FC
:1008000002C000E81FEF0093830010938400089556
:1008100000918300B09180000B0F10918400B09183
:1008200081001B1F20E03091840033230AF42A95B5
:10083000B09182002B1F1AF4203F40F00AC02F30E5
:1008400008F407C00FEF1FEF2FE003C000E010E037
:1008500020EF30916300B0919B003B1718F43230C9
:1008600030F009C0B0918400BB235AF004C0B091AD
:100870008400BB2332F40093800010938100209306
:10088000820008952091D70000918300000F1091FD
:100890008400111F46DF11232AF40038BFEF1B0725
:1008A00040F009C00F37120508F405C00FE710E04B
:1008B00002C000E81FEF002352F0B0916200B01BAD
:1008C0000B2F18F0013008F00AC001E008C00095B5
:1008D0000F5FB09162000B0F08F001C00FEF0093A3
:1008E000850008952091D800009181001091820028
:1008F00018DF11232AF40130BFEF1B0740F009C0B5
:100900000F3F120508F405C00FEF10E002C001E030
:100910001FEF112352F0B0918500B01B0B2F18F080
:10092000013008F00AC001E008C000950F5FB091E7
:1009300085000B0F08F001C00FEF009363000895CE
:100940000FEF71FD1EC0B091D300BB23D1F0B09169
:100950007B00BB23B1F00FEF10917B00B7DEF89462
:10096000B091730072FDB5E00B9F112D002D7894AE
:10097000112309F00FEFB0919E000B1710F40091B6
:100980009E0000939D00089500917A0010917B00D5
:1009900000541140B0919D0010F4BA9501C0B39578
:1009A00011F0B0939D00089500C008952091B50006
:1009B000B6B1B6FDFBCF04B115B1B6B1BF77B6B9CC
:1009C000B091AA00B395B093AA00B83060F120921C
:1009D000AA00B091D200BB2321F1112329F0B091DC
:1009E000AB00BF3F61F009C0B091AB000B1739F00D
:1009F00020F4BB2321F0BA9502C0B395E1F3009136
:100A00009B00B093AB00B03050F400ECB03038F441
:100A100000E8B03020F400E4B03008F400E00093C7
:100A20009B007F7E089510919B00B0E11B0F08F49E
:100A30001FEF10939B00B091B400B43081F000918F
:100A40009B00B0916300B01B10F400916300B09163
:100A50009D000B1708F00B2F502E00936400B091EF
:100A6000AA00B73009F47061089502E3F894B091D8
:100A7000D9000B9F012D000C001F7894B0919B00B2
:100A80000B1710F000919B0000936100009363002E
:100A9000502E0093640000939E00089520927A00E7
:100AA000B0EFB0937B000895F8940CB51DB520917C
:100AB0007400789430917500609076000093750012
:100AC00010937600031B160971FD03C077FD80C0EB
:100AD00028C070907700209377002709222319F00F
:100AE0000FEF1FEF0EC08090780090907900309348
:100AF00078006092790000917500109176000819D5
:100B0000190920917A0030917B0036952795020FC4
:100B1000131F10F40FEF1FEF00937A0010937B0068
:100B20002BC020917A0030917B003901B4E08B2EEC
:100B3000B2E09B2E343040F08A949A94383020F002
:100B400072FD02C08A949A94769467948A94E1F72D
:100B500026193709992021F0169507959A94E1F7FF
:100B6000200F311F20937A0030937B0028F43FEF51
:100B700030937A0030937B00323008F4706871FF54
:100B800002C0B3E00DC0B091C40000917100023802
:100B900038F0B395003A08F0B395B63008F0B5E0F8
:100BA0009B2EB4E08B2E10917B0000917A0024E004
:100BB000169507952A95E1F70819120928F0B02F24
:100BC000B250B12FB20910F402E010E0980126C033
:100BD00020917A0030917B00390176946794669475
:100BE000669466942619320906950695200F321DE3
:100BF00020937A0030937B00323008F07F7704E056
:100C0000369527953695279526952695201B10F025
:100C1000223008F422E089019090C40060FDFECFEC
:100C2000E0908B00F0908C006160B9B7B061B9BF03
:100C3000380177FD41C07694679400938B00109340
:100C40008C00B92DB330E1F0B0FD04C0060D171DC6
:100C5000930106C0000F111F0250120922E030E07C
:100C6000B92DB33068F020938D0030938E0000933F
:100C70008700109388006092890070928A003AC0C1
:100C800000938D0010938E0020938700309388008E
:100C90006092890070928A0071FF0DC0BFE0B0932E
:100CA0008D0020928E00B093890020928A00B0932C
:100CB0008B0020928C001EC0669400938B00B92D8F
:100CC000B33091F0B0FD03C0060D262D03C0000F18
:100CD000025022E0B92DB33038F020938D000093FC
:100CE00087006092890006C000938D0020938700E2
:100CF0006092890000917C0002FD0350013031F4C4
:100D000095FD0CC0B2E0B06CB7B90BC0023021F455
:100D1000B3E0B06CB7B905C095FDF4CFB4E0B06CEA
:100D2000B7B90091A200000F10F4BBE60B270093A7
:100D3000A20060FDFECFB2E0B0936E006160B9B773
:100D4000B061B9BFB72FB670D1F020917A00309161
:100D50007B00369527953695279571FF02C0B0E444
:100D60003B0FF8940CB51DB5020F131F1BBD0ABD38
:100D70006160B0E1B8BFB9B7B061B9BF7894089508
:100D8000686020927D0020E066FD20E206C0686079
:100D900020927D0020E266FD20E001E011E077FD79
:100DA00011C0B72FB67009F0677F14E100917B0086
:100DB000069509F403950F3008F00FE071FF02C0AB
:100DC00004E114E160FD0FC0B0917D00BB2359F038
:100DD00071FF06C0B0916E00BA95B0936E0011F429
:100DE00070624FC0ABDFB0B7B77FB0BFB8B1B0B7BC
:100DF000B860B0BFB0917D00B395B0937D00B8B13D
:100E000077FD06C0B1E071FDB3E0BA95F1F7B8B176
:100E1000B072B21709F02AC071FF05C0039501171F
:100E200008F00A95CFCF63FD05C00395011708F0C0
:100E3000B4CFC8CF677FF8943CB56DB470907A009A
:100E4000B0917B00770CBB1F08F4BFEF770CBB1F82
:100E500008F4BFEF370D6B1E6BBC3ABD6160B0E1AB
:100E6000B8BFB9B7B061B9BF789497CFB0916D00F2
:100E7000B13008F492CF63FD90CF0A9509F0A2CF6C
:100E80007F7D20918D0030918E00F894B0E1B8BF45
:100E90000CB51DB5020F131F1BBD0ABDE0908700E6
:100EA000F09088006160B9B7B061B9BF7894B72F8E
:100EB000B67039F0B0916D0072FFB395B0936D00CC
:100EC00009C075FF07C066FD05C063FD03C0BF9183
:100ED000BF91FBC4089500E063FF01C001E0F894F6
:100EE00010917100B7E01B9F212D102D7894200FD9
:100EF00026951795269517952695179510937100A9
:100F0000183718F4B8E7B093710000917100B091F0
:100F100072000B1720F0606190989198939860FD93
:100F2000FECFE0908900F0908A006160B9B7B061AF
:100F3000B9BF0895B2E095FD0AC0F894B0937C0063
:100F40009798959A62FF01C0939A7894F4C0F894A8
:100F5000B0937C009798949A62FF01C0909A78941D
:100F6000EAC0B3E082FF24C095FD11C002E0F8940E
:100F7000B0937C00ECE7F0E00093B1009398949874
:100F800062FF02C0919A01C0979A7894D4C002E09F
:100F9000F894B0937C00ECE7F0E00093B1009098F7
:100FA000959862FF02C0919A01C0979A7894C3C045
:100FB00095FD0BC0F894B0937C00E6E6F0E09398C2
:100FC00062FF01C0919A7894B6C0F894B0937C0007
:100FD000E6E6F0E0909862FF01C0919A7894ABC089
:100FE000B4E095FD0AC0F894B0937C009598949A6B
:100FF00062FF01C0919A78949EC0F894B0937C00EF
:101000009498959A62FF01C0919A789494C0B5E043
:1010100082FF24C095FD11C001E0F894B0937C00DC
:10102000E2E7F0E00093B1009198979862FF02C068
:10103000909A01C0959A78947EC004E0F894B09399
:101040007C00E6E8F0E00093B1009198979862FF89
:1010500002C0939A01C0949A78946DC095FD0BC01C
:10106000F894B0937C00E0E6F0E0919862FF01C054
:10107000909A789460C0F894B0937C00ECE6F0E02D
:10108000919862FF01C0939A789455C0B6E095FD9F
:101090000AC0F894B0937C009498979A62FF01C0BC
:1010A000909A789448C0F894B0937C009598979A59
:1010B00062FF01C0939A78943EC0B1E082FF24C0E1
:1010C00095FD11C004E0F894B0937C00E6E8F0E0F0
:1010D0000093B1009098959862FF02C0939A01C066
:1010E000949A789428C001E0F894B0937C00E2E7E9
:1010F000F0E00093B1009398949862FF02C0909A38
:1011000001C0959A789417C095FD0BC0F894B093E0
:101110007C00ECE6F0E0909862FF01C0939A78942E
:101120000AC0F894B0937C00E0E6F0E0939862FF88
:1011300001C0909A78946F7E08952FE530E0F90110
:101140002092B10090989198939895989798949838
:101150006B7F0895A2EBB0E009E00D9309E00D93D9
:1011600004E00D930FEF0D9303E00D930FEF0D933C
:101170000AE00D9301E00D9301E00D9301E00D9362
:10118000AEEBB0E001E00D930FEF0D930D930D93D7
:101190000D930D9303E00D930FEF0D930FEF0D9350
:1011A0000D9305E20D9300ED0D9308E20D9300E51C
:1011B0000D9304E00D930FEF0D9302E00D9300E00B
:1011C0000D930AE70D930FEF0D9300E00D9301E0EF
:1011D0000D9300E00D9303E00D9300E00D9308954F
:1011E0002091B9008B7FB091BA00B33019F09F7D88
:1011F000B1FD90629F7BB091BB00B1FD9064223045
:1012000011F0886001C0877F08950A95E00FF21DF4
:10121000B4910895ECE1F0E00091B200F6DFB093F4
:10122000D700ECE1F0E00091B300EFDFB093D8001D
:10123000EAE2F0E00091B800E8DFB093D900009155
:10124000B800023008F402E000937300B091CE00C1
:101250000FEFB23009F400EAB33009F402E800936A
:101260007200E8E3F0E00091D500CFDFB093A0007A
:10127000089508952091C8003091C900B091BA0036
:10128000B33009F43E5097FF02C020E03FEFB32F88
:10129000B21B6B2EB25810F4B2E86B2E00E003952F
:1012A000609EB12DBD57D8F30093AC0008959068AF
:1012B000E1DFBFD9BED920E030E0B0E16B2EB5D977
:1012C000B09196002B0F321D6A94C9F7B4E03695A1
:1012D0002795BA95E1F7822E9F77CCDF0895F89491
:1012E000E3E0F0E0B9E0B7BFB491B078C1F3F894AF
:1012F000A895B1B5B861B1BDB0E0B1BDB4E0BEBFB5
:10130000BFE5BDBF1ADFB0E0B8BBB0E1B7BBB0E02E
:10131000B5BBB0E0B4BBB0E0B2BBBBEBB1BB222409
:10132000A0E0B0E02D92AA31E9F7A0E6B0E00FEF1F
:101330002D920A95E9F7B1E0B093A2000BDF01D33B
:10134000B7E0B06CB7B9B6B1B460B068B6B90091E7
:10135000CA000093AD00B1E0B0936A00F8946DD973
:1013600077D967D978D965D979D963D9F8940AEF4B
:101370001AEFA0B396FDA095A2FF1FC01A95C9F75A
:101380000A95B1F7E0E0FCE1B591B43E39F4B591CE
:10139000B03E21F4B591BF3F09F40CC0E0E0F395F5
:1013A000F395B591B83F49F4B591B43931F4B5919D
:1013B000BA3A19F4EE27F695099412DF2BDF59DFBC
:1013C00059DF0091CA000093AD00B7DEB2E0B3BFB1
:1013D000B2E0BEBDB2E0B5BDB1E5B8BFB9BFB0B710
:1013E000B77FB0BFB8B1B0B7B860B0BF1CD9789400
:1013F000DBDA20927000B3E096FDB2E0B5BFB0E456
:10140000BBBFBB27B064BABF8D7F17D9626033E022
:101410002CE0B0919500BB2321F42CE03A9509F41F
:10142000A5CF07D980FFA2CF8E7FB0919600B230B2
:1014300078F3B92FBF710091980000939700B09393
:101440009800B01729F72A9521F76D7FB3E096FD34
:10145000B2E0B5BFBB27B064BABF8D7FB091D400F6
:10146000BB2321F48062B92FB0709B2F8F7B209219
:101470006700E1D885FF05C0B0916700BA3008F079
:101480008064D3D802E085FF01C000E0B0919600EF
:10149000B017B8F3F894DCD8DBD8DAD87894CDD884
:1014A00020928600B091BA00B33009F47DC0BDD857
:1014B000B091BE00B13008F477C0B0916A00B1308D
:1014C00008F472C085FD18C0B0919600BF3F08F4C3
:1014D0006BC0F894C6D87894AED8B0919600B1306D
:1014E000C0F7F894B5D8A3D8B3D87894A4D8B0915D
:1014F0009600BF3FB0F3E6C2B3E09B2E9068F8942D
:10150000B9DE789498D8F8949F77B4DE80909600EE
:10151000B0919600BF37789408F44EC084D8F89400
:10152000A0D878949A9451F7C2DEB82DB093C90030
:1015300084D8F8949AD27894BAE09B2E9068F89464
:1015400099DE789478D8F8949F7794DE809096000E
:10155000B0919600BF37789478F765D8F89478D82A
:1015600066D876D878949A9449F7A1DEB82DBB5FF7
:10157000B093C8000B2F1091C900125810F0100B37
:1015800020F4B2E80B0F0093C90057D8F89406D2A4
:101590007BD2789450D8F8946DDE7894B091960010
:1015A000BF3F08F48FCF8EC200919600B0918600A5
:1015B0000B1710F0009386003ED801E0B091BA00FE
:1015C000B35009F405E0B0919600B01708F06ACF67
:1015D000F89447D846D845D878942FD820926A00F6
:1015E00020926B0020926C00B0916B00B395B09389
:1015F0006B00BF3F71F5B0916C00B395B0936C0078
:10160000B091CC0009E1BA9559F002E3BA9541F0E6
:101610000DE7BA9529F00AEFBA9511F020926C0007
:10162000B0916C00B017A8F088DDFDD7B0916C00C8
:10163000BA95B0936C0020926B00B091CB00B09340
:10164000AD00F8940ED87894B091CA00B093AD0074
:10165000F2D7EDD7B0916800BB2319F485FF01C024
:1016600085CE01E085FD01C006E0B0919600B0177F
:1016700008F4BACFB091BA00B35009F0DCD7B091FA
:101680006800BB2309F472CEF89457DD2092610004
:101690002092620020926300522C209264002092DB
:1016A000A1007894B091B700BB0FB0939F00209237
:1016B0007E0020927F002092800020928100209264
:1016C00082002092AA0060E070E020927100B8E0F1
:1016D000B093AA007061A7D7B7E074FDB7E0B06C13
:1016E000B7B9B6B1B068B064B6B9B6B1B6FDFDCFA2
:1016F00004B115B1B6B1BF77B6B9112309F00FEF38
:101700000093AB0053D9B8E0B093AA00706168DDD4
:10171000F894BFEFB0939B00A8D9B0916100B0934B
:101720009B00B0939C00B0939D007894B1E0B0937F
:101730006100B09363005B2EB0936400B093A4008B
:10174000B0919A00B093A300B091BA00B33019F4ED
:101750009F7D87FD90627160726020926D0096DCC3
:10176000ACDC9CD9A1D99AD99FD998D910DBFBD7E9
:10177000B2DBE0DB99D904DB65FD2ED877FFE0D83A
:1017800077FD02D9A8DBEDDB8FD901DB65FD40D801
:10179000A2DB26DC89D9F4DA65FD74D89CDB37DC62
:1017A00083D9F5DA65FD9ED896DB70DC7DD9E8DA61
:1017B000B7E074FDB7E0B06CB7B9B6B1B068B0646B
:1017C000B6B989DB7ADC70D9F1D871FF24C0B09149
:1017D0009E00B0939B00B0939C00B0919A00B09390
:1017E000A300B1E0B093A40018E12CE0B0916D002B
:1017F000B11758F07D7F746020936F00B0919E0008
:10180000B0939B00B0939D0006C0B0919600B1309C
:1018100008F0ACCF64C072FF15C066FD13C0B09174
:101820006F00BA9519F47B7F7860A0CFB0936F00FA
:10183000B0919600B13008F099CFB091BA00B330B2
:1018400009F04DC020927000B09199000AEF1091FC
:10185000D600112309F003E0B01708F040C085FF5F
:1018600004C0B0916800BB23D1F1B091BA00B3308D
:1018700081F495FD03C087FD04C00BC087FF01C044
:1018800008C066FD06C06064B0919E00B0939B00E6
:1018900082CF00EF66FF05C0B0919E00B0939B0021
:1018A00000E2B0917B00B01708F460CF66FF17C06C
:1018B0006F7B9F7D87FD90627460B2E1B0936F0093
:1018C000B0919E00B0939B0051CFB0917000B39542
:1018D000B0937000B0919600BB2309F002C0209233
:1018E0007000F8942ADC8090B900B2E0B093B9009F
:1018F00077DC8092B90020926100209262002092F1
:101900006300522C2092640020929F0060E070E0FF
:10191000789491D612DC0091D600002319F0909AA9
:10192000919A939AB7E0B06CB7B9B6B1B460B068A9
:10193000B6B985FF05C0B0917000B43008F016CD7F
:101940004FCEEDE0F0E023D0053509F01BC0EEE00E
:10195000F0E01DD00A3A09F015C03AE0A2EBB0E081
:10196000E3E0F0E014D00D9331963A95D9F739E1E0
:10197000AEEBB0E0EFE0F0E00AD00D9331963A958F
:10198000D9F702C0E7DB0AD0E8E2F0E00895E19978
:10199000FECFEEBBFFBBE09A0DB308951ED03AE038
:1019A000A2EBB0E0E3E0F0E00D910FD031963A9574
:1019B000D9F739E1AEEBB0E0EFE0F0E00D9105D002
:1019C00031963A95D9F712D00895E199FECF0DBB23
:1019D000EEBBFFBBE29AE19A0895EDE0F0E00FEF75
:1019E000F4DFEEE0F0E00FEFF0DF0895EDE0F0E07F
:1019F00005E5EBDFEEE0F0E00AEAE7DF089530917D
:101A0000AE000091AF00313011F40093B2003230DB
:101A100011F40093B300333011F40093B400343068
:101A200011F40093B600353011F40093B80036304D
:101A300011F40093C400373011F40093B90038302A
:101A400011F40093D500393011F40093CE003A30F0
:101A500011F40093BA003B3011F40093BB000895D9
:101A600025E0EBD52A95E9F70895F2D5F4D5F6D51A
:101A7000F8D5DDD5EDD5EFD5F1D5F3D5D8D5E8D569
:101A8000EAD5ECD5EED50895ECD5E8D5E4D5E0D58A
:101A9000CED5E7D5E3D5DFD5DBD5C9D5E2D5DED5C3
:101AA000DAD5D6D508958090AE009090AF00D0D50D
:101AB000CFD5CED5BCD58A94D1F7D3D5B8D59A9405
:101AC000E1F70895F894D1DF7894CADFC9DFB1E077
:101AD000B093AE00B1E0B093AF002092B000F894A4
:101AE000E2DF7894B5E06B2E70909600A6D5B091A9
:101AF00096007B16C9F7B13018F0BF3F40F107C020
:101B00007EDFF8944BDFB1DFB8E0B1BDA9DF6A94A6
:101B100059F7B091B000B395B093B000B33008F46A
:101B2000DECF9EDFB091AF00B395B093AF00F894D5
:101B3000B091AE00BA95EEE3F0E0EB0FF21D049128
:101B400078940395B091AF00B01708F4C6CF88DF42
:101B500087DFB091AE00B395B093AE00B091AE0008
:101B6000BC3008F4B7CFF6DAF89418DFB8E0B1BDAE
:041B700077DFB5CB9B
:00000001FF
